:100000000C9417060C942C290C9459290C943F0637
:100010000C943F060C94C20C0C943F060C943F06C3
:100020000C943F060C943F060C943F060C943F063C
:100030000C943F060C943F060C943F060C943F062C
:100040000C9486290C943F060C94402D0C947B2D27
:100050000C943F060C943F060C943F060C943F060C
:100060000C943F060C943F065F1C661C661C5F1CCC
:10007000661C661C661C661C661C661C661C661C70
:10008000661C661C661C661C661CD41B661C661CF3
:10009000661C661C661C3E1B661C661C661C661C79
:1000A000661C661C661C661C661C661C661C661C40
:1000B000661C661C661CE01BE01BE01BE01BE01BD3
:1000C000E01BE01BE01BE01B661C661C661C661C3C
:1000D000661C661C3E1BDF1BDF1BDF1BDF1B661C59
:1000E000F01BF81B001C081C101C181C201C281CD2
:1000F000321C3C1C461C501C831B431B661C661C8C
:10010000661C661CD41B661C661C661C661C661C72
:10011000661C661C661CDE1BDE1BDE1BDE1B661CF3
:10012000F01BF81B001C081C101C181C201C281C91
:10013000321C3C1C461C501C831B431B661C661C4B
:10014000661C661CD41B971C971C971C971C971C3D
:10015000971C971C971C971C971C971C971C971C07
:10016000B71DB71DB71DB71DB71DB71DDE1CE81C99
:10017000F21CFC1C621D6C1D7A1D8B1D281E981E16
:10018000691E6E1E731E781E7D1E821E871E981E9F
:10019000921EB125C625D225DB25E8250E2616267A
:1001A00039262626456E746572206D656E752E2E75
:1001B0002E00546F67676C6564206D6963726F50C1
:1001C000504D00546F67676C656420696E76657288
:1001D0007465642050504D2100546F67676C6564EE
:1001E000205458206D7574696E672100546F6767DD
:1001F0006C65642074656C656D657472792100505E
:10020000726F746F636F6C206572726F72207769A2
:1002100074682052580054696D656F757420776852
:10022000656E20636F6E6E656374696E6720746FB0
:1002300020525800507265737320616E79206B658F
:100240007920746F2063616E63656C00436F6E6E1E
:10025000656374696E6720746F2052582C20706F2C
:100260007765722075702074686520525820287751
:100270006974682062696E6420706C7567206966B5
:10028000206E6F74207573696E6720616C77617979
:10029000732062696E642900546F67676C6564201F
:1002A00027696D6D656469617465206F757470751B
:1002B000742700546F67676C65642027736C6176E0
:1002C00065206D6F64652700546F67676C656420F7
:1002D00027616C776179732062696E642700546FBF
:1002E00067676C65642050504D206368616E6E6571
:1002F0006C206C696D6974005365742052535349C6
:1003000020696E6A656374696F6E206368616E6EE2
:10031000656C2028303D3D64697361626C6529001D
:100320005365742050504D206D696E696D756D2058
:1003300073796E630053657420626561636F6E202C
:10034000696E74657276616C0053657420626561D4
:10035000636F6E2064656C6179005365742062651B
:1003600061636F6E206672657175656E6379206971
:100370006E20487A3A20303D64697361626C652C66
:100380002050783D504D52206368616E6E656C2040
:10039000782C2046783D465253206368616E6E6526
:1003A0006C2078005365742050574D2073746F7023
:1003B0002064656C61792028302064697361626C07
:1003C00065642C20312D323535203D3D20302E31D5
:1003D00073202D2035306D696E29005365742050CF
:1003E000504D2073746F702064656C6179202830E3
:1003F0002064697361626C65642C20312D3235355F
:10040000203D3D20302E3173202D2035306D696E1A
:100410002900536574206661696C736166652064A8
:10042000656C61792028302064697361626C656451
:100430002C20312D323535203D3D20302E3173209A
:100440002D2035306D696E29002A2A2A2A2A2A2A67
:100450002A2A2A2A2A2A2A2A2A2A2A2A2A2A2A2AFC
:100460002A2A2A2A2A2A0052582041636B656420CE
:100470002D2072657665727420737563636573737E
:1004800066756C21002A2A2A2A2A2A2A2A2A2A2A36
:100490002A2A2A2A2A2A2A2A2A2A2A2A2A2A2A2ABC
:1004A0002A2A002A2A2A2A2A2A2A2A2A2A2A2A2AD6
:1004B0002A2A2A2A2A2A2A2A2A2A2A2A2A2A2A2A9C
:1004C0000052582041636B6564202D207570646173
:1004D0007465207375636365737366756C21002A98
:1004E0002A2A2A2A2A2A2A2A2A2A2A2A2A2A2A2A6C
:1004F0002A2A2A2A2A2A2A2A2A2A2A2A0056616CE1
:1005000069642063686F69636573206172653A206E
:100510005B315D2D5B31365D20286368616E6E65F1
:100520006C20312D31362900536574206F7574703D
:10053000757420666F7220706F727420005B585D56
:100540002061626F7274206368616E6765732061F9
:100550006E64206578697420525820636F6E6669F6
:1005600067005B535D207361766520736574746901
:100570006E677320746F205258005B525D20726565
:10058000766572742052582073657474696E67734F
:1005900020746F2064656661756C747300557365B3
:1005A000206E756D62657273205B312D445D207421
:1005B0006F206564697420706F727473205B452DC1
:1005C000515D20666F722073657474696E67730085
:1005D000202D20726563656976657220636F6E6693
:1005E0006967757261746F722C207278207377203E
:1005F000000A0A6F70656E4C52536E672000536597
:10060000742073657269616C2062617564726174D3
:10061000653A200056616C69642063686F696365A0
:10062000733A2031202D20342B34202F2032202DDE
:100630002038202F2033202D20382B34202F203419
:10064000202D203132202F2035202D2031322B3407
:10065000202F2036202D203136005365742043682A
:10066000616E6E656C20636F6E6669673A20005339
:1006700065742044617461726174652028302D3284
:10068000293A200053657420486F70206368616EBA
:100690006E656C7320286D61782032342C20736570
:1006A0007061726174656420627920636F6D6D6141
:1006B00073292076616C69642076616C756573209E
:1006C000312D3235353A2000536574206368616EF0
:1006D0006E656C2073706163696E672028783130B5
:1006E0006B487A293A200053657420524620706F77
:1006F0007765722028302D37293A20005365742001
:100700005246206D616769632028686578292065F5
:100710002E672E20307844454144463030443A20FC
:10072000005365742062617365206672657175653A
:100730006E63792028696E20487A293A20005B5A36
:100740005D20656E74657220726563656976657299
:1007500020636F6E66696775726174696F6E20756C
:1007600074696C79005B465D20646973706C6179B3
:100770002061637475616C206672657175656E6366
:100780006965732075736564005B525D2063616CFD
:1007900063756C6174652072616E646F6D206B654A
:1007A0007920616E6420686F70206C697374005BDF
:1007B000495D207265696E697469616C697A65204A
:1007C00073657474696E677320746F20736B6574DE
:1007D00063682064656661756C7473005B585D20A6
:1007E000726576657274206368616E6765732061F7
:1007F0006E642065786974206D656E75005B535D6D
:1008000020736176652073657474696E67732074F4
:100810006F20454550524F4D20616E6420657869C8
:1008200074206D656E7500557365206E756D62651B
:100830007273205B302D395D20746F20656469749C
:1008400020706172616D657465727300202D205394
:10085000797374656D20636F6E6669677572617414
:10086000696F6E000A0A6F70656E4C52536E672096
:10087000005129204F7574707574206265666F721F
:1008800065206C696E6B20283D465329203A200074
:10089000502920536C617665206D6F646520286552
:1008A00078706572696D656E74616C293A20004FCD
:1008B000292054696D65642042494E4420617420AA
:1008C0007374617274757020203A20004E29205094
:1008D000504D206F7574707574206C696D69746506
:1008E0006420202020203A200044495341424C45B6
:1008F00044004D292050504D205253534920746FCD
:10090000206368616E6E656C202020203A20004CC8
:10091000292050504D206D696E696D756D20737979
:100920006E63202875732920203A200044495341E2
:10093000424C4544004B29204661696C73616665F1
:1009400020626561636F6E20696E74762E20283197
:100950002D32353573293A20004A29204661696CC9
:100960007361666520626561636F6E2064656C61AA
:10097000792028302D323535203D3E20313073200E
:100980002D203135306D696E293A200049292046E5
:1009900061696C7361666520626561636F6E206674
:1009A00072712E203A200048292050574D20737430
:1009B0006F702064656C6179202020202020203A0F
:1009C000200047292050504D2073746F70206465BB
:1009D0006C6179202020202020203A200046292008
:1009E0004661696C736166652064656C617920207D
:1009F00020202020203A200050574D206368616E4F
:100A00006E656C200066756E6374696F6E3A2000C7
:100A10002920706F72742000506F776572546F7761
:100A2000657200445446205548462033322D626991
:100A3000742031306368004F70656E4C52536E679E
:100A40005258206D696E6920342F36636800466CF9
:100A50007974726F6E2F4F72616E676552582055B0
:100A600048462038636800525820747970653A20EF
:100A70000044697361626C656400487A00203D3D02
:100A8000200043616C63756C617465642070616300
:100A90006B657420696E74657276616C3A200042F1
:100AA00029204D6963726F202868616C6629205087
:100AB000504D202020203A00412920496E76657251
:100AC0007465642050504D20696E20202020203A0B
:100AD000003029204D7574652062757A7A65722020
:100AE000286D6F73746C79293A0039292053657227
:100AF00069616C2062617564726174653A00736D3E
:100B0000617274506F7274004672536B7900547244
:100B1000616E73706172656E740044697361626CBA
:100B200065640038292054656C656D657472793A86
:100B300020202020202020003729204368616E6E6D
:100B4000656C20636F6E6669673A20200036292045
:100B500044617461726174652028302D32293A2015
:100B6000202000352920486F70206368616E6E6513
:100B70006C733A2020202020003429204368616EC5
:100B80006E656C2073706163696E673A2020003374
:100B90002920524620706F7765722028302D372922
:100BA0003A202020003229205246206D6167696377
:100BB0003A202020202020202020003129204261BE
:100BC0007365206672657175656E63793A202020C1
:100BD0000000000000240027002A0000000000257B
:100BE0000028002B0000000000230026002900043C
:100BF00004040404040404020202020202030303C4
:100C000003030301020408102040800102040810BD
:100C1000200102040810200000000700020100006B
:100C2000030406000000000000000000232F112430
:100C30001FBECFEFD8E0DEBFCDBF13E0A0E0B1E034
:100C4000E8E8F0E602C005900D92A839B107D9F79F
:100C500016E0A8E9B3E001C01D92AB35B107E1F79A
:100C60001CE0CEE2DCE004C02297FE010E941F30AF
:100C7000CC32D107C9F70E94682F0C9442300C94F3
:100C80000000A0E0B0E0E7E4F6E00C94EE2FEC0109
:100C9000A880B980CA80DB80A114B104C104D1044A
:100CA00041F484E2A82E89EDB82E8BE5C82E87E0AA
:100CB000D82EC601B5012DE133EF41E050E00E948E
:100CC000CB2F27EA31E440E050E00E94772F7B01F0
:100CD0008C01C601B5012DE133EF41E050E00E94E7
:100CE000CB2FCA01B9012CEE34EF4FEF5FEF0E941A
:100CF000772F6E0D7F1D801F911F97FF04C06150DD
:100D0000704080409048688379838A839B839B01ED
:100D1000AC015F77B901CA01CDB7DEB7EAE00C9448
:100D20000A300E944106089581EB92E00E9441063C
:100D300008956093B1027093B2028093B3029093CE
:100D4000B4020895A0E0B0E0E8EAF6E00C94E72FE2
:100D5000EC012B016A016115710519F0FB0191830A
:100D60008083C114D10449F0C6010297839728F00B
:100D700020E030E040E050E0DCC0A9908A2D90E017
:100D80000E943730892BC9F7FDE2AF1621F4A990F4
:100D90003324339405C08BE2A81609F4A9903324B8
:100DA000C114D10421F0E0E1CE16D10411F5F0E335
:100DB000AF1669F48881883711F0883541F4A9802D
:100DC000229682E0382A20E1C22ED12C12C0C11412
:100DD000D10479F4E0E3AE1659F199E9E92E99E9E5
:100DE000F92E99E9092F99E1192F8AE0C82ED12C03
:100DF0003AC0FAE0CF16D10491F080E1C816D104D0
:100E000029F0E8E0CE16D104F9F415C0BFEFEB2EBF
:100E1000BFEFFB2EBFEF0B2FBFE01B2F24C0A9E9B4
:100E2000EA2EA9E9FA2EA9E90A2FA9E11A2F1BC077
:100E3000F8E0CF2ED12CEFEFEE2EEFEFFE2EEFEFFE
:100E40000E2FEFE11E2F0FC09601442737FD40956E
:100E5000542F6FEF7FEF8FEF9FEF0E94A92FC901F3
:100E6000DA017C018D0120E030E040E050E060E0FC
:100E70003601882477FC8094982C70EDB72EBA0C3C
:100E8000F9E0FB1570F48A2D81548A3118F499EC3D
:100E9000B92E06C08A2D81568A3148F589EAB82EC6
:100EA000BA0C8B2D90E08C159D050CF56F3FE9F089
:100EB000E216F30604071507B8F0CA01B901A40148
:100EC00093010E94772F9B01AC018B2D90E0A0E055
:100ED000B0E0280F391F4A1F5B1F281739074A0740
:100EE0005B0710F061E001C06FEFA990C6CF41141D
:100EF000510451F0662311F0219703C031FE04C064
:100F00002297F201D183C08330FE07C050954095EF
:100F1000309521953F4F4F4F5F4F67FF0AC082E2E8
:100F200090E090935A06809359062FEF3FEF4FEFD2
:100F30005FEFB901CA01CDB7DEB7E1E10C94033030
:100F4000FC0188279927E89421912032E9F3293080
:100F500010F02E30C8F32B3241F02D3239F4689462
:100F600004C00E94F507820F911D219120532A3061
:100F7000C0F31EF4909581959F4F089548E953E082
:100F80000E94C3070895009731F4DA018D919C9176
:100F9000009709F40EC0DC01FB013D912191222351
:100FA00019F03217C9F3FACF332331F4DA011D9265
:100FB0001C928827992708951197AF93BF93FB013F
:100FC0003D912191321771F4332321F48827992719
:100FD000119702C01E921196FA01A193B0839F91BE
:100FE0008F910895222369F7EACF7AE0979F902D99
:100FF000879F802D910D1124089580919A0381304F
:1010000019F482E080939A0380919A03833019F453
:1010100084E080939A030895E3E0F0E089E0809310
:101020005700849190E08670863009F491E0892F12
:1010300008951F93182F0E940C08882379F09FB7FA
:1010400081E08093A105F894A89588E180936000E1
:1010500010936000112309F0A8959FBF1F91089578
:10106000382F20E080913305909134058227932713
:1010700040E061E270E19C01220F331F97FF04C042
:10108000C9018627972701C0C9014F5F483099F7EA
:101090009093340580933305089587E38093D003BC
:1010A00080E092ECA1E0B0E08093D1039093D20372
:1010B000A093D303B093D40387E08093DD0380E053
:1010C00091EAACEBB3E38093D5039093D603A0935E
:1010D000D703B093D80385E08093DE038DEE9EEFB7
:1010E000ADEABEED8093D9039093DA03A093DB03BE
:1010F000B093DC03AFEDB3E080E090E0863010F019
:10110000E0E004C0FC01EF57FC4FE081ED93019655
:101110008831910599F782E08093F7038AE0809304
:10112000F803089580E09EECADEEB4E380939D0358
:1011300090939E03A0939F03B093A00380E090E060
:10114000A0E0B0E58093A1039093A203A093A30332
:10115000B093A403E5EAF3E080E081938F5F8031F0
:10116000E1F708958436910520F4BC0180E090E019
:1011700025C08E3B910550F48A559040BC0180E01B
:1011800090E02AE030E040E050E016C0823D91055A
:1011900050F4845B9040BC0180E090E024E630E0B5
:1011A00040E050E009C08D5C9040BC0180E090E0E0
:1011B00028E532E040E050E00E94772F24E630E05E
:1011C00040E050E00E94772F089590E08C599F4FA7
:1011D0000E94B2080895DC019896EC91F0E0E77067
:1011E000F070E758FC4F808108958F929F92AF92E4
:1011F000BF92CF92DF92EF92FF920F931F938C01D9
:101200000E94EB08D80197962C9130E043E150E022
:10121000249FF001259FF00D349FF00D1124EB5415
:10122000FD4F80809180A280B38090E00F96AA2726
:1012300097FDA095BA2FBC01CD0120E43FE14DE719
:1012400050E00E94772FA50194010E94A92F690107
:101250007A0180ED97E0A0E0B0E0C80ED91EEA1E4A
:10126000FB1ED80198968C91887181F060E07EEE2B
:101270008AEB9BE0A50194010E94A92F28513C4FC5
:101280004F4F5F4FC20ED31EE41EF51E87EE93E054
:10129000A0E0B0E0C80ED91EEA1EFB1EC701B601D1
:1012A00028EE33E040E050E00E94A92FCA01B901C6
:1012B00028EE33E040E050E00E94772F1F910F911D
:1012C000FF90EF90DF90CF90BF90AF909F908F9066
:1012D00008958F3F910509F010F480E0089522E011
:1012E0008030920710F481E008958050934010F010
:1012F00083E0089582E00895CF92DF92FF920F93EA
:101300001F93CF93DF93F82FEB016A01182F1695E7
:10131000E0E088819981D6018C938A819B81119626
:101320008C9311978C819D8112968C9312978E814C
:101330009F8113968C931397288139814A815B8111
:101340006C817D818E819F819295990F990F907C00
:10135000832F8370982B852F8370880F880F982B8D
:10136000872F83708295807F982B14969C9385E0BD
:1013700090E0C80ED91E2896EF5F1E1750F6F0FFBA
:1013800021C0888199810E946909F82E8A819B81F8
:101390000E946909182F8C819D810E946909082F7C
:1013A0008E819F810E946909F294FF0CFF0C70EC02
:1013B000F7221295107F1F29182B000F000F012B09
:1013C000D6010C93DF91CF911F910F91FF90DF9089
:1013D000CF90089523E08032920718F420E030E0A7
:1013E00026C023E0883E920748F49C012F513340E9
:1013F00054E0369527955A95E1F719C027E0803DCE
:10140000920720F49C012C5D334011C028E08839FC
:10141000920718F02FEF33E00AC09C01285C374098
:1014200044E0369527954A95E1F72D503C4FC90188
:1014300008958C30910548F49C0174E0220F331F0D
:101440007A95E1F7285D3C4F17C023E0843F92076F
:1014500020F49C0124523C4F0FC024E080309207BE
:1014600018F020E938E008C09C012657334F64E0AB
:10147000220F331F6A95E1F7C90108959C01369543
:10148000279525753575821B930B9C0136952795FD
:10149000369527952373337383739373280F391FFE
:1014A000C901E4E096958795EA95E1F7820F931FCD
:1014B0008F709F7021E031E0AC01429FC001439FDB
:1014C000900D529F900D1124892F0895882339F093
:1014D0005F980000289A00005F9A000008955F98C6
:1014E0000000289800005F9A000008955F9A0000AD
:1014F00083B15F98000090E096958795817008957C
:101500000F931F93082F5C9A5F985C9810E0802FD0
:1015100080780E94660A000F1F5F1830C1F75F983D
:101520001F910F9108958F770E94800A08950F935D
:101530001F93082F10E0802F80780E94660A000F0A
:101540001F5F1830C1F75F981F910F9108950F9397
:101550001F935F9880E000E0182F110F0E94760A19
:10156000810F0F5F0830C1F71F910F9108950E94FE
:10157000930A0E94A70A5C9A08951F93162F806809
:101580000E94800A812F0E94970A5C9A1F910895F9
:101590001F931091D9031827E0EDF3E0E80FF11D38
:1015A00089E767850E94BD0A8DE3612F0E94BD0A0D
:1015B00082E4612F0E94BD0A1F91089586E20E9475
:1015C000B70A08950F931F938C018CE1F801648191
:1015D0000E94BD0A8DE1F80165810E94BD0A8EE17D
:1015E000F80166810E94BD0A80E2F80167810E94CD
:1015F000BD0A81E2F80160850E94BD0A82E2F8011D
:1016000061850E94BD0A83E2F80162850E94BD0ADD
:1016100084E2F80163850E94BD0A85E2F8016485D1
:101620000E94BD0A8AE2F80165850E94BD0A8EE625
:10163000F80166850E94BD0A8FE6F80167850E9461
:10164000BD0A80E7F80160890E94BD0A81E7F801C0
:1016500061890E94BD0A82E7F80162890E94BD0A81
:101660001F910F910895EF92FF920F931F93CF93C5
:10167000DF937B018C01603028E372072CE982073D
:101680002CE1920728F520E836E948E950E00E946D
:10169000A92FE9016897B90180E090E020E839E6D8
:1016A00047E65FEF0E94772F6E0D7F1D801F911F11
:1016B00032E0660F771F881F991F3A95D1F721E70F
:1016C00032E040E050E00E94A92F890180E421C06F
:1016D00020E03DE241E351E00E94A92FE901689733
:1016E000B90180E090E020E033ED4EEC5EEF0E9427
:1016F000772F6E0D7F1D801F911F660F771F881F2C
:10170000991F21E732E040E050E00E94A92F8901B3
:1017100080E69E012F71622F680F85E70E94BD0A47
:1017200086E7612F0E94BD0A87E7602F0E94BD0AED
:10173000CDB7DEB7E6E00C940E30682F8DE60E9440
:10174000BD0A08959F92AF92BF92CF92DF920F93FE
:10175000DF93CF9300D000D0CDB7DEB7982E83E0D3
:101760000E94B70A8093F90384E00E94B70A80932D
:10177000FA0386E060E00E94BD0A87E061E00E9413
:10178000BD0A89E06FE70E94BD0A8AE065E00E9419
:10179000BD0A8BE062E10E94BD0A8CE065E10E9417
:1017A000BD0A8DE06DEF0E94BD0A8EE060E00E94F0
:1017B000BD0A992019F084E193E008C08091F703F5
:1017C00023E1829FC00111248B549D4F0E94E20AA5
:1017D00080E36CE80E94BD0A82E36FE00E94BD0ACC
:1017E00083E362E40E94BD0A84E36AE00E94BD0ACA
:1017F00085E36AE20E94BD0A86E36DE20E94BD0AAB
:1018000087E364ED0E94BD0A88E360E00E94BD0AA0
:1018100089E360E00E94BD0A992049F065E8A62EA0
:1018200061ECB62E61ECC62E6EEDD62E08C0A090EF
:10183000D903B090DA03C090DB03D090DC030AE355
:101840008D2D9927AA27BB2789839A83AB83BC83D5
:10185000802F69810E94BD0A802F8B5F69810E9461
:10186000BD0ADC2CCB2CBA2CAA240F5F0E3341F717
:1018700083E46FEF0E94BD0A84E46FEF0E94BD0A0B
:1018800085E46FEF0E94BD0A86E46FEF0E94BD0AF7
:10189000992019F08DE666E003C08DE66091DD03C6
:1018A0000E94BD0A89E760E00E94BD0A8AE7609154
:1018B000DE030E94BD0A83E760E00E94BD0A84E760
:1018C00060E00E94BD0A992029F060E071EA8CEB8B
:1018D00093E308C06091D5037091D6038091D7033C
:1018E0009091D8030E94330B0F900F900F900F90A0
:1018F000CF91DF910F91DF90CF90BF90AF909F90ED
:10190000089587E061E00E94BD0A8EE764E20E94CC
:10191000BD0A88E063E00E94BD0A88E060E00E94A2
:10192000BD0A87E065E00E94BD0A85E062E00E9492
:10193000BD0A83E00E94B70A8093F90384E00E9405
:10194000B70A8093FA030895582F40919E04842F7C
:1019500090E0FC01EF70F0709F012F5F3F4F74E04B
:10196000959587957A95E1F72817390751F0E25751
:10197000FB4F5083842F8F5F8F70407F842B809329
:101980009E0408951F920F920FB60F921124EF92AA
:10199000FF920F931F932F933F934F935F936F93F8
:1019A0007F938F939F93AF93BF93EF93FF93E090B9
:1019B000A103F090A2030091A3031091A40389B1A5
:1019C000A8019701207430704070507090E063E07F
:1019D000969587956A95E1F7A0E0B0E081709070E8
:1019E000A070B070281739074A075B0709F46AC06E
:1019F000209184003091850010928500109284001F
:101A00008091C104882309F05DC0E5FC02C03695D1
:101A1000279589E0253C3807C8F180914703A80144
:101A200097011CE156954795379527951A95D1F75B
:101A3000211531054105510521F421E030E040E058
:101A400050E090E0A0E0B0E0281739074A075B07B4
:101A5000D0F4809147038F3FB1F020E00EC0E22F19
:101A6000F0E0EE0FFF1FDF01AE53BB4F8D919C9155
:101A7000E95DFC4F918380832F5F80914703281796
:101A800070F31092C004109247031CC082E02D3BFB
:101A90003807A8F080914703803188F410914703FC
:101AA000C9010E94EA09E12FF0E0EE0FFF1FEE539B
:101AB000FB4F918380831F5F1093470303C08FEF19
:101AC00080934703FF91EF91BF91AF919F918F91C9
:101AD0007F916F915F914F913F912F911F910F9146
:101AE000FF90EF900F900FBE0F901F90189583E01E
:101AF000809380008AE1809381008FEF9FEF909325
:101B000089008093880010926F0088E080936D00B8
:101B1000E8E6F0E080818460808308956F3018F0FB
:101B200086958058089589E0689F802D1124089536
:101B3000882319F460E071E002C063E071E087E39C
:101B400096E00E942B2D0895A0E0B0E0EAEAFDE0C7
:101B50000C94F02F182F0E94DC299B01AC0180917E
:101B60002D0590912E05A0912F05B09130056901AA
:101B70007A01C81AD90AEA0AFB0AD701C6018958AC
:101B80009341A040B04010F010922C0520932D05F9
:101B900030932E0540932F05509330052091C104BA
:101BA000822F81508230E8F580912C05882309F43A
:101BB0004FC1813011F482E0BCC1803108F035C1E1
:101BC000E82FF0E0EE53FB4F10838F5F80932C05DE
:101BD000803109F0B0C1A4ECB4E0213039F41196A1
:101BE000EC911197E695E6958C9109C08D919C91A9
:101BF0001197E92FE695E695E69596958795E0315C
:101C000040F4F0E090E0EE0FFF1FE95DFC4F9183A0
:101C100080831092C004129684E0A23DB807E9F6D2
:101C20008AC1233009F004C180912C05882321F456
:101C30001F3009F080C10CC1883130F4E82FF0E08A
:101C4000EF53FB4F108374C1883109F0EEC01123AC
:101C500009F0EBC0C0E0D0E00BE010E0DE0163E093
:101C6000AA0FBB1F6A95E1F7C09FB001C19F700D1D
:101C7000D09F700D1124FB01EE53FB4F8081218119
:101C8000922F977095958795FD01EE0FFF1FE95DE7
:101C9000FC4F91838083FB01ED53FB4F30813695E0
:101CA000369536952181422F4295440F407E842FF0
:101CB000832B269526952695922F97709595879537
:101CC000FD01EE0FFF1FE75DFC4F91838083FB0159
:101CD000EC53FB4F80818295869586958370418178
:101CE000942F990F990F292F282B429546954695A9
:101CF000437082818170880F880F382F342B35957F
:101D00002795FD01EE0FFF1FE55DFC4F318320831A
:101D1000FB01EA53FB4F308136952181422F4795D5
:101D200044274795842F832B2695922F977095955E
:101D30008795FD01EE0FFF1FE35DFC4F91838083CC
:101D4000FB01E953FB4F308132953F702181422FD7
:101D50004295407F842F832B22952F70922F97706E
:101D600095958795FD01EE0FFF1FE15DFC4F918377
:101D70008083FB01E853FB4F8081881F8827881FE1
:101D80004181942F990F292F282B441F4427441F4A
:101D900082818370880F382F342B35952795FD016C
:101DA000EE0FFF1FEF5CFC4F31832083FB01E653F6
:101DB000FB4F3081369536952181422F4295440F55
:101DC000440F407C842F832B26952695922F977065
:101DD00095958795AA0FBB1FFD01ED5CFC4F918384
:101DE000808365537B4FFB012081229526952770C8
:101DF0004181342F330F330F330F832F822B942FD6
:101E000092959695977095958795AB5CBC4F11967A
:101E10009C938E932196C230D10509F01FCF8091FB
:101E2000D80483FD02C01092C00410922C0583C018
:101E3000243009F080C040912C05442359F4183A0D
:101E4000B1F4109234051092330588EA0E943008EC
:101E500081E06FC0413019F41093310504C0423065
:101E600031F410933205812F0E9430085DC06091DB
:101E70003205262F30E0220F331FE42FF0E0C90196
:101E800002968E179F0734F0433268F7E154FB4FF8
:101E90001083E9CF2D5F3F4F4091330550913405BA
:101EA000E217F30749F4912F80E048275927509310
:101EB00034054093330538C0812F90E04817590707
:101EC00089F580913105813069F5613118F080E143
:101ED00080933205D0903205F2ECEF2EF4E0FF2E25
:101EE00000E010E01BC0F701D081C0E0818190E0EC
:101EF0008C2B9D2BE3E096958795EA95E1F70E9460
:101F0000EA09F801EE0FFF1FE95DFC4F9183808322
:101F10000F5F1F4F82E090E0E80EF91E0D1518F3D9
:101F20001092C00410922C0580912C05882319F082
:101F30008F5F80932C05CDB7DEB7E8E00C940C30B2
:101F4000FF920F931F93CF93DF93182F092FF62E35
:101F50008EE30E94BD0A212F302FC901EC0110E051
:101F600005C08FE769910E94BD0A1F5F1F15C8F366
:101F700085E064E00E94BD0A83E00E94B70A809376
:101F8000F90384E00E94B70A8093FA030E94DC29D7
:101F90006093FB037093FC038093FD039093FE0317
:101FA00087E069E00E94BD0A81E080939A03CDB783
:101FB000DEB7E5E00C940F300E94A00F80919A03E9
:101FC0008130D9F40E94DC292091FB033091FC037D
:101FD0004091FD035091FE03621B730B840B950B24
:101FE000605A76488140904040F4E8CF87E396E01D
:101FF00067E071E00E942B2D089580919A03813053
:10200000A9F3089587E396E06EE70E94E32E089512
:10201000A0E0B0E0EEE0F0E10C94EF2F6C0187E37C
:1020200096E06EE70E94E32E760100E010E0C0E04B
:10203000D0E0B0E2BB2E0AC00830110521F49E01A9
:102040002095F60120870894E11CF11CF7016081BE
:10205000862F8D57823040F487E396E06DE70E942B
:10206000E32EF70160816B2587E396E00E94E32E63
:102070000115110551F0F70180819E01280F311DD6
:10208000C32FDD27C20FD31FD0700F5F1F4F093042
:10209000110591F6CDB7DEB7E9E00C940B30A9E05D
:1020A000B0E0E5E5F0E10C94F62F382FE62F8091B3
:1020B000A30490E0019664E270E00E94962F982FAE
:1020C0008093A30488E9898380E18A83913071F049
:1020D000913028F0923099F09330E1F416C085E009
:1020E0008B8381EF8C832F5F2D8317C09B8381EFC0
:1020F0008C8384E6489FC00111249D830EC084E038
:102100008B8381EF8C833D8308C09B8381EF8C831D
:10211000ED8303C00E94021004C0CE0101960E940C
:1021200008102996E2E00C9412300F931F93CF937E
:10213000DF93182F092F87E396E06EE70E94E32EC6
:10214000212F302FC901EC0110E000E288818D576A
:10215000823040F487E396E06DE70E94E32E8881A9
:102160008027888387E396E069910E94E32E1F5FB2
:10217000193061F787E396E06EE70E94E32EDF9166
:10218000CF911F910F910895A9E0B0E0EAECF0E142
:102190000C94F62F382F8091A304882379F48EEFC6
:1021A00089833A836B83842F90E0959587958C8300
:1021B0002D83198618861F821E822FC040919E048F
:1021C000842F90E09C012F70307054E09595879596
:1021D0005A95E1F78217930721F18DEF89831A82CF
:1021E0001B82DE01149620E008C0E257FB4F80817D
:1021F0008D93405F2F5F263069F0842F90E0FC01C3
:1022000034E0F595E7953A95E1F78F709070E8170F
:10221000F90759F740939E042A83CE0101960E9444
:1022200095108091A30490E0019666E070E00E9412
:10223000962F8093A3042996E2E00C9412309F928B
:10224000AF92BF92CF92DF92EF92FF920F931F93C4
:10225000B82EA62ED42EC22E902E0E94DC297B01F1
:102260008C0180918D0420919F043091A0044091B5
:10227000A1045091A2048823B1F0D801C701821BA8
:10228000930BA40BB50B815E9E42A040B04020F1A1
:102290002C2DDC1408F42D2D8B2D6A2D422F292D89
:1022A0000E944F1011C0D801C701821B930BA40BD1
:1022B000B50B81539547A040B04070F08B2D6A2D2F
:1022C0004D2D2C2D0E94C410E0929F04F092A0048A
:1022D0000093A1041093A2041F910F91FF90EF901F
:1022E000DF90CF90BF90AF909F90089587E396E0E6
:1022F000609100040E94E32E08951F93182F87E336
:1023000096E0612F0E94E32E809100048127809344
:1023100000041F9108951F93192F0E947D11812F92
:102320000E947D111F910895DF92EF92FF920F930B
:102330001F93D82E7B011092000407E316E0C8011A
:1023400065EB0E94E32EC80162E60E94E32E8D2D0C
:102350000E947D11C7010E948B111F910F91FF9068
:10236000EF90DF900895E82FF0E0E456FC4FE18510
:10237000E03158F4F894F0E0EE0FFF1FE95DFC4FF8
:102380000190F081E02D78940DC0E03129F0E13129
:1023900029F0E0E0F2E006C082E101C083E10E94A2
:1023A000302BFC01CF01089589E060E00E94612A92
:1023B00088E061E00E94612A87E061E00E94612A72
:1023C00082E060E00E94612A84E061E00E94612A6C
:1023D0000895892B19F08AE061E002C08AE060E08C
:1023E0000E94CD2A0895A0E2B0E0E9EFF1E10C945B
:1023F000EE2F8CE00E94B70A882379F587E396E0F8
:1024000063E171E00E942B2D2D9A80E00E94A20BC7
:102410000E94810C2D9821C087E396E00E94AA2E8D
:10242000482F8091C104882321F0842F0E94A40D9D
:1024300014C080912A05E82FF0E031969F012F719A
:10244000307031978091290590E02817390729F0DD
:10245000E050FB4F408320932A0587E396E00E94DB
:10246000702E892BC9F680919A03843009F08EC0B2
:102470000E94DC296093B0047093B1048093B2048D
:102480009093B304611571058105910561F481E0B4
:1024900090E0A0E0B0E08093B0049093B104A093EA
:1024A000B204B093B3048091BC049091BD048160E8
:1024B0009093BD048093BC0483E080939A038FE7DC
:1024C0000E94930A07EF14E00E94A70AF801819383
:1024D0008F01F5E000301F07B9F74091E2048091C9
:1024E000F704282F30E0842F90E08227932786FF7F
:1024F00040C080E448274093E204C901887390708B
:10250000C89709F510E014C01F5F8091F803E12F10
:10251000F0E084FF06C0E950FB4F80810E94A40CCC
:1025200007C0E950FB4F87E396E060810E94E32EED
:10253000212F30E08091F70490E08770907082172F
:10254000930714F716C02F733070232B91F48091EA
:10255000F8048093B4048091F9048093B6048091C8
:10256000FA048093B7048091FD048093BE04109216
:10257000BF0480912B05813019F482E080932B05F4
:1025800080912B05833011F410922B050E94DC29D9
:102590005B016C018091B8049091B904A091BA04D8
:1025A000B091BB040097A105B105C9F08601750182
:1025B000E81AF90A0A0B1B0BD801C701885B9B407C
:1025C000A040B04060F00E94DE0A8093B5041092F3
:1025D000B8041092B9041092BA041092BB0480EDB2
:1025E00093E00E94F5082091AC043091AD04409135
:1025F000AE045091AF0486017501E21AF30A040B90
:10260000150BE616F7060807190708F424C1A0926F
:10261000AC04B092AD04C092AE04D092AF04A895C1
:102620008091C0048830A0F08091A1039091A20312
:10263000A091A303B091A403FCE1B695A79597954B
:102640008795FA95D1F70097A105B10509F0A2C1C8
:102650008091C0048F5F8093C004E090B004F0903C
:10266000B1040091B2041091B304E114F104010526
:10267000110511F180ED93E00E94F508AE18BF0836
:10268000C00AD10A6A157B058C059D0588F48091E6
:10269000A10384FD04C080ED97E00E94E91110922F
:1026A000B0041092B1041092B2041092B30404C0AA
:1026B00080E090E00E94E9119091E204907C909378
:1026C000E20400912A05109129050117B1F18091CA
:1026D0002B05823091F590589093E20480ED93E0C1
:1026E0000E94EB08893010F048E002C0482F4150AA
:1026F00030E013C03F5FA32FB0E0812F90E0FC01DA
:10270000E050FB4F2081FD01EE51FB4F2083A05E86
:10271000BA4F2C930196182F1F71341710F410170D
:1027200049F710932905832F895C9091E204892B46
:102730008093E204309320051AC020912B052430A9
:10274000D1F490912005E1E2F5E0A3EEB4E0292F69
:1027500030E02E0F3F1F02C081918D93E217F307E7
:10276000D9F7995C8091E204982B9093E20483E07E
:1027700080932B0536C08091A704823059F4916074
:102780009093E2042D9A05EA13E07E010894E11C7F
:10279000F11C10C09093E2042D98222319F481E0DB
:1027A00080932B0580912B05833069F784E080931B
:1027B0002B05E9CFF80181918F010E94B311F70138
:1027C000819391937F01F3E0053B1F0799F7809177
:1027D000F8038770BE016F5F7F4F43EE54E00E94A5
:1027E0007C092C9A2091A5042223A1F09091DD036D
:1027F000992381F08091A6048F5F8093A604815075
:10280000821729F41092A604892F815001C0892FC4
:102810000E949D0B8091A4040E94C80A80ED93E061
:102820000E94EB08682F82EE94E00E94A00FE091D6
:10283000A404EF5FE093A404E83131F0F0E0E0534A
:10284000FC4F8785882339F41092A40404C02D9A84
:1028500089E08093C0048091F803887171F18091C0
:102860009A03823051F58091BC049091BD04880F89
:10287000991F9093BD048093BC0483E080939A03D6
:102880000E94810C0E94DC296093B8047093B90403
:102890008093BA049093BB0461157105810591057D
:1028A00061F481E090E0A0E0B0E08093B804909300
:1028B000B904A093BA04B093BB048091F80384FFD9
:1028C0001EC08091BC049091BD048E7F0E943E0A80
:1028D000182F8091B4046091BE040E948E0D082FC1
:1028E0008091B504612F0E948E0D282F8091B6042F
:1028F0006091B704402F00919B030E941F112C98F8
:102900008091A7048130D1F0813020F0823009F02D
:1029100047C034C08BE00E94002B892B09F040C0D7
:1029200081E08093A7040E94CE296093A80470934D
:10293000A9048093AA049093AB0432C08BE00E9458
:10294000002B892B21F50E94CE292091A8043091DB
:10295000A9044091AA045091AB04621B730B840B31
:10296000950B695E734080409040D0F082E0809388
:10297000A70480ED97E00E94E91112C08BE00E944D
:10298000002B892B69F080E090E00E94E911109201
:10299000A70406C08091C004883009F059CF57CFF2
:1029A000A096EAE00C940A308AE061E00E94612A75
:1029B0008AE060E00E94CD2A08951F93182F0E949C
:1029C000DC2960939F047093A0048093A1049093EA
:1029D000A20410938D04112329F440E855E260E02D
:1029E00070E004C040E051EE60E070E087E396E004
:1029F0000E94E92D1F910895ACE1B0E0E2E0F5E11D
:102A00000C94EE2F0E94DC297B018C0181E00E9456
:102A1000A20B84E7A82E6E010894C11CD11CB3E060
:102A2000BB2EA982C60161E00E94DC0FB0929A031E
:102A30000E94810C6AEF70E080E090E00E94022A20
:102A400080919A03833009F07DC087E396E00E946D
:102A5000702E892B09F076C00E94DC296E197F093F
:102A6000800B910B6058734C894C914008F06AC000
:102A7000D8CF8FE70E94930A0E94A70A843509F0F5
:102A80005CC089830E94A70A182F00E010932404D9
:102A9000009323040E94A70A080F111D1093240419
:102AA000009323040E94A70A809322040E94A70A8D
:102AB00080932104813108F040C0FF2407C00E94A8
:102AC000A70A0F5F1B4FF8018083F3940F2D10E0CE
:102AD0008091210490E0880F991F0817190778F357
:102AE00080E78983CE01019661E00E94DC0F83E0DC
:102AF00080939A030E94810C62E370E080E090E092
:102B00000E94022A80919A038330A9F08FE70E94E5
:102B1000930A0E94A70A803581F4898305EB13E0AC
:102B20000E94A70AF80181938F01F3E0003D1F077F
:102B3000B9F781E003C082E001C083E06C96EAE06F
:102B40000C940A3080919A03833009F092CFF3CF2E
:102B500083E00E94B70A8093F90384E00E94B70AD9
:102B60008093FA0387E061E00E94BD0A6AE070E0AA
:102B700080E090E00E94022A0E94810C00000895EB
:102B80000F931F93082F17C02D9A64E670E080E022
:102B900090E00E94022A2D9864E670E080E090E0C8
:102BA0000E94022A1F5F101778F36CE271E080E048
:102BB00090E00E94022A10E0F6CF482F392F25E03E
:102BC0000DC0F999FECF1FBA842F932F92BD81BDFE
:102BD00060BD0FB6F894FA9AF99A0FBE215059F0D9
:102BE000F999FECF842F932F92BD81BDF89A80B5BD
:102BF000681739F7089582E00E94C0150895A0E093
:102C0000B0E0E5E0F6E10C94E72F482E562ECC24F8
:102C1000DD24EE24FF2488249924C0E0D0E076E46B
:102C2000372E04C0CC24DD2455245394442069F469
:102C300080919B03839DE00111246CE9E62E63E003
:102C4000F62E59E1852E912C1DC021E0421671F41B
:102C500080919B03839DE00111246B9640EDE42E4F
:102C600043E0F42E39E2832E912C0CC032E043165F
:102C700049F42BE9E22E23E0F22E91E0892E912CEB
:102C8000C8E1D1E03E016C0C7D1C1092340510921D
:102C90003305E3011BC0552059F4F999FECFD2BD8D
:102CA000C1BDF89A80B5F701E00FF11F808307C01E
:102CB000F701E00FF11FCE0160810E94DD150E0DBE
:102CC0001F1DF80180810E94300821969E0126195F
:102CD000022F10E008151905F0F2CE015520D9F4A5
:102CE000F999FECFD2BDC1BDF89A20B5F999FECFB2
:102CF0002196D2BDC1BD2197F89A80B590E0B22E41
:102D0000AA248A299B29209133053091340528175C
:102D1000390759F487CF2196609134050E94DD155B
:102D2000CE01609133050E94DD1580E291E0C80E6E
:102D3000D91E91EEC91692E0D90608F477CF852DF9
:102D4000CDB7DEB7E1E10C94033080E061E00E9492
:102D5000FF1581E061E00E94FF15089582E061E0C7
:102D60000E94FF15089582E060E00E94FF158091A7
:102D70009B03843020F010929B030E94AE160895AE
:102D80001F93182F0E94B31680919B03811731F077
:102D9000143020F410939B030E94AE161F910895E7
:102DA00010928B0485E6E6E2F4E0DF011D928A953D
:102DB000E9F708951F93182F8F3711F08830E1F548
:102DC000E0918B04EE2309F455C0E150E0938B04AD
:102DD000F0E0EA5DFB4F108287E396E06DE00E9431
:102DE000E32E10E00AC0E12FF0E0EA5DFB4F87E33D
:102DF00096E060810E94E32E1F5F80918B0418177C
:102E000090F387E396E060E20E94E32E87E396E08A
:102E10006DE00E94E32E10E00AC0E12FF0E0EA5DD1
:102E2000FB4F87E396E060810E94E32E1F5F809155
:102E30008B04181790F31CC08B3119F40E94D01624
:102E40001FC08D30E9F08A30D9F080918B04843630
:102E500088F487E396E0612F0E94E32E80918B0433
:102E6000E82FF0E0EA5DFB4F10838F5F80938B04C7
:102E700080E007C087E396E067E00E94972BF8CFD9
:102E800081E01F9108951F93CF93DF93CFEDD3E09F
:102E900010E03BC087E396E062E271E00E94282DDB
:102EA00087E396E0612F4AE050E00E94A52C87E37B
:102EB00096E06FE271E00E94282D699170E080E059
:102EC00090E02091DE0330E040E050E00E94772F58
:102ED00020E137E240E050E00E94772FDC01CB0197
:102EE0004091D5035091D6036091D7037091D803D8
:102EF000480F591F6A1F7B1F87E396E02AE030E0E6
:102F00000E946C2C1F5F183119F08881882311F6FC
:102F1000DF91CF911F910895EF92FF920F931F932E
:102F2000882339F487E396E061E77AE00E94B52BC5
:102F30003BC090E00E94B20824E630E040E050E060
:102F40000E94A92F122F032FF42EE52E622F732F2C
:102F5000842F952F2AE030E040E050E00E94A92F16
:102F600087E396E0BA01A9012AE030E00E945D2CD7
:102F700087E396E06EE20E94972B612F702F8F2DD2
:102F80009E2D2AE030E040E050E00E94A92FAB01E6
:102F9000BC0187E396E02AE030E00E945D2C87E3E5
:102FA00096E063E70E94C92B1F910F91FF90EF906D
:102FB0000895FF920F931F93CF93DF9387E396E0DB
:102FC00067E67AE00E94762B8091B503813041F468
:102FD00087E396E06EE47AE00E94B52BFF246DC093
:102FE000823029F487E396E067E37AE0F5CF843016
:102FF00029F487E396E063E27AE0EECF853071F75B
:1030000087E396E068E17AE0E7CFCF2DD0E0C930E2
:10301000D1051CF06F2D685C02C06F2D6F5C87E3DB
:1030200096E00E94972B87E396E060E17AE00E94A9
:10303000762BBE016F5F7F4F87E396E04AE050E05A
:103040000E94012D87E396E065E07AE00E94762BEE
:103050008E010B541C4FD8011196EC91E032F8F41C
:1030600087E396E068EF79E00E94762BF801818192
:10307000803130F087E396E063E371E00E94282D11
:10308000CB54DC4F698170E06F7070706F5F7F4F61
:1030900087E396E04AE050E00E94142D0DC0F0E076
:1030A000EF70F070EE0FFF1FE75BFC4F60817181E6
:1030B00087E396E00E942B2DF39480912204F8166A
:1030C00008F4A3CF87E396E06DED79E00E94762BBC
:1030D0008091CD030E948C1787E396E062EC79E043
:1030E0000E94762B8091CE030E948C1787E396E096
:1030F00067EA79E00E94762B8091CF030E948C17BB
:1031000087E396E06CE879E00E94762B4091C50356
:103110005091C6036091C7037091C80341155105D2
:103120006105710539F187E396E02AE030E00E94FD
:103130006C2C87E396E069E579E00E94762B80911C
:10314000C9030E94E508AB01BC0187E396E02AE0D1
:1031500030E00E946C2C87E396E065E379E00E9402
:10316000762B87E396E06091CA034AE050E00E9424
:10317000B72C06C087E396E06CE279E00E94B52B9D
:1031800087E396E06FE079E00E94762B6091CB03B5
:103190007091CC0387E396E04AE050E00E94912CC6
:1031A00087E396E062EF78E00E94762B6091C4039B
:1031B000603450F470E06F5F7F4F87E396E04AE041
:1031C00050E00E94142D06C087E396E069EE78E097
:1031D0000E94B52B87E396E06CEC78E00E94762B9A
:1031E0008091C30380FD03C065E371E002C069E321
:1031F00071E087E396E00E942B2D87E396E06FEA6B
:1032000078E00E94762B8091C30382700E94980D13
:1032100087E396E060E978E00E94762B8091C30313
:1032200084700E94980D87E396E061E778E00E9441
:10323000762B8091C30388700E94980DCDB7DEB7BE
:10324000E5E00C940F301F93CF93DF9387E396E074
:103250006BEB7BE00E94762B4091D5035091D60317
:103260006091D7037091D80387E396E02AE030E0BD
:103270000E946C2C87E396E065EA7BE00E94762B47
:103280004091D9035091DA036091DB037091DC0324
:1032900087E396E020E130E00E946C2C87E396E023
:1032A0006FE87BE00E94762B87E396E06091DD0378
:1032B0004AE050E00E94B72C87E396E069E77BE0A4
:1032C0000E94762B87E396E06091DE034AE050E0AF
:1032D0000E94B72C87E396E063E67BE00E94762BA2
:1032E000CFEDD3E010E012C0112331F087E396E078
:1032F0006DE371E00E94282D87E396E069914AE032
:1033000050E00E94A52C1F5F183119F08881882396
:1033100059F787E396E00E949F2B87E396E06DE4E0
:103320007BE00E94762B87E396E06091F7034AE00A
:1033300050E00E94B72C87E396E068E37BE00E94B0
:10334000762BE091F803F0E0E770F070EE0FFF1FCE
:10335000E759FC4F6081718187E396E00E942B2D35
:1033600087E396E063E27BE00E94762B8091F8038E
:1033700090E0887190708830910589F089309105CE
:103380001CF4892B39F01BC08031910569F04897F6
:10339000B1F40FC087E396E06AE17BE00EC087E3FB
:1033A00096E06EE07BE009C087E396E068E07BE0B2
:1033B00004C087E396E06EEF7AE00E94B52B87E3C6
:1033C00096E06AEE7AE00E94762B4091D10350910C
:1033D000D2036091D3037091D40387E396E02AE08F
:1033E00030E00E946C2C87E396E061ED7AE00E9469
:1033F000762B8091A10380710E94980D87E396E05F
:1034000068EB7AE00E94762B8091A10380740E9481
:10341000980D87E396E06FE97AE00E94762B809121
:10342000A10380720E94980D87E396E062E87AE03B
:103430000E94762B80ED93E00E94F508AB01BC0161
:1034400087E396E02AE030E00E945D2C87E396E077
:103450006DE77AE00E94762B80ED93E00E94F508FC
:103460009B01AC0160E472E48FE090E00E94A92F20
:1034700087E396E0BA01A9012AE030E00E945D2CC2
:1034800087E396E06AE77AE00E94B52BDF91CF915F
:103490001F910895EF92FF920F931F937C0107E312
:1034A00016E0C8016F2D70E04AE050E00E94802CC9
:1034B000C8016EE20E94972BB70184E0769567956C
:1034C0008A95E1F76F707070C8014AE050E00E9481
:1034D000802CC8016EE20E94972B8FE0E822FF2427
:1034E000C801B7014AE050E00E94802C1F910F9163
:1034F000FF90EF9008950F931F93CF93DF93209148
:1035000025042F3FA9F587E396E061EF75E00E945F
:10351000762B83E793E00E944A1A87E396E060EDFA
:1035200075E00E94762B80912304909124040E94E0
:103530004A1A87E396E06DE975E00E94B52B87E3B0
:1035400096E06AE775E00E94B52B87E396E062E6B5
:1035500075E00E94B52B87E396E06DE375E00E946D
:10356000B52B87E396E00E949F2B0E94D91769C074
:1035700012160CF066C0332727FD30958091220487
:1035800090E0821793070CF45CC087E396E068E252
:1035900075E00E94762B60912504772767FD709572
:1035A00087E396E04AE050E00E94142D87E396E01E
:1035B0006DEF74E00E94762B08E210E03AC0C12F54
:1035C000D0E0CC0FDD1FCF5FDB4F288130E0809152
:1035D0002504992787FD909501972817390741F50C
:1035E00087E396E06FE371E00E94282D87E396E081
:1035F000602F4AE050E00E94A52C87E396E063E448
:1036000071E00E94282DE981F0E0EF70F070EE0F7C
:10361000FF1FE75BFC4F6081718187E396E00E94AA
:10362000282D87E396E067E471E00E94282D0F5F64
:103630001F5F80912104181710F287E396E00E9423
:103640009F2BDF91CF911F910F910895ACE1B0E0D6
:10365000ECE2FBE10C94F02F282F809125048F3FA2
:1036600009F03BC1822F90E0FC013A97EF36F1055B
:1036700008F02CC1EC5CFF4F0C941D3087E396E002
:1036800069E471E0A7C087E396E065E571E00E9418
:103690002B2D85E78983DE011296E5EBF3E08BE1C4
:1036A00001900D928150E1F7CE0101966CE10E94EC
:1036B000DC0F0E94810C83E080939A0368EC70E039
:1036C00080E090E00E94022A80919A03843009F001
:1036D000FDC08FE70E94930A0E94A70A898385355F
:1036E00009F0F4C087E396E06FED74E00E94B52B1B
:1036F00087E396E061EC74E00E94B52B87E396E0E7
:1037000063EA74E0ACC087E396E06DE671E00E9486
:103710002B2D89E68983CE01019661E00E94DC0FA2
:103720000E94810C83E080939A0368EC70E080E053
:1037300090E00E94022A80919A03843009F0C6C06A
:103740008FE70E94930A0E94A70A89838E010E5F69
:103750001F4FBDE1EB2EF12CEC0EFD1E0E94A70ABF
:10376000D8018D938D01AE15BF05C1F7A5EBB3E070
:10377000FE0132968BE101900D928150E1F7898133
:10378000893409F0A3C087E396E065E874E00E94FD
:10379000B52B87E396E067E674E00E94B52B87E3DC
:1037A00096E069E474E05BC087E396E067E871E067
:1037B0000E942B2D8EEF8093250488C02052275025
:1037C000922F905380912204891738F487E396E072
:1037D00066E971E00E942B2D79C0909325046FC09B
:1037E00084E18093250487E396E062E174E037C0CA
:1037F00085E18093250487E396E06BED73E02FC0AD
:1038000086E18093250487E396E064EA73E027C0AD
:1038100087E18093250487E396E06AE573E01FC0A3
:1038200088E18093250487E396E069E473E017C09C
:1038300089E18093250487E396E065E373E00FC098
:103840008AE18093250487E396E060E273E007C095
:103850008BE18093250487E396E068EF72E00E9495
:10386000B52B34C087E396E06EED72E00E94B52B75
:103870008091C30391E01DC087E396E068EC72E09D
:103880000E94B52B8091C30392E013C087E396E0BA
:1038900063EB72E00E94B52B8091C30394E009C0F2
:1038A00087E396E068E972E00E94B52B8091C3033C
:1038B00098E089278093C3038FEF809325040E94AB
:1038C0007B1A04C087E396E00E94AA2E87E396E065
:1038D0000E94702E892BB1F762C1822F0E94DA16E6
:1038E000882309F45CC180918B04882321F48FEF35
:1038F000809325044CC186E294E060E070E040E0F3
:1039000050E00E94A2069B01AC0160912504862F25
:10391000992787FD9095A92FB92FFC013197EB319D
:10392000F10508F024C1ED55FF4F0C941D30E62F32
:10393000FF27E7FDF0958091220490E08E179F0706
:103940000CF415C1DA01C9010197A109B1098097E9
:10395000A105B10548F0A8E2FA2E00E010E06F01E1
:103960000894C108D10825C0EB54FC4F822F815028
:103970008083E5C0612F70E0660F771F6F5F7B4F1C
:10398000FB01808190E08C159D0591F48F2D90E0D6
:10399000A0E0B0E082179307A407B50741F4F60151
:1039A000EB54FC4FDB0111968C91818301E0F39481
:1039B0001F5F809121041817E8F2BFC02F3F310527
:1039C0004105510511F008F0D2C02093CD03B7C0D6
:1039D0002F3F31054105510511F008F0C8C0209373
:1039E000CE03ADC02F3F31054105510511F008F060
:1039F000BEC02093CF03A3C080912604806280378D
:103A000019F587E294E060E070E040E050E00E9449
:103A1000A2069B01AC01DC01CB010197A109B10910
:103A20000897A105B10508F0B5C0CA01B90124ED98
:103A300030E340E050E00E94772F9B01AC012A5E0A
:103A40003C4A4A46554E24C0863611F587E294E03A
:103A500060E070E040E050E00E94A2069B01AC01F3
:103A6000DC01CB010197A109B1090797A105B105B7
:103A700008F090C0CA01B90128EA31E640E050E000
:103A80000E94772F9B01AC01245E3C434E46544E6E
:103A9000211531054105510561F0DA01C901805058
:103AA0009447AB48B24381509A45A246B24008F0D1
:103AB0005EC02093C5033093C6034093C703509361
:103AC000C8033DC02F3F31054105510511F008F0F5
:103AD0004EC02093C90333C0DA01C9010197A1097F
:103AE000B1098F3F9105A105B10508F040C02093B1
:103AF000CA0325C0DA01C901845C9940A040B040E6
:103B00008D549D41A040B04030F43093CC032093BD
:103B1000CB0301E001C000E021153105410551054D
:103B200011F48FEF07C0213431054105510528F408
:103B3000822F81508093C40302C00023C1F0809182
:103B40008C048823D1F48091D9039091DA03A09159
:103B5000DB03B091DC030196A11DB11D8093D90355
:103B60009093DA03A093DB03B093DC0306C087E3F2
:103B700096E068EA71E00E942B2D0E94D0168FEF2C
:103B80008093250487E396E06AE00E94C92B0E9497
:103B90007B1A05C021E030E040E050E07ECF6C961B
:103BA000E8E00C940C3087E396E06CE472E00E944D
:103BB000B52B87E396E064E372E00E94B52B87E3C0
:103BC00096E00E94702E892B31F087E396E00E94E8
:103BD000AA2E0E94261B0E94FC14823019F083300A
:103BE00069F405C087E396E066E172E004C087E30C
:103BF00096E06FEF71E00E94B52B08958FEF8093F0
:103C0000250410928C040E947B1A0CC087E396E076
:103C10000E94702E892B31F087E396E00E94AA2E35
:103C20000E94261B809125048E3F81F70895809184
:103C30002504992787FD9095A92FB92FFC0131966E
:103C4000EB30F10508F074C0E254FF4F0C941D30C6
:103C500087E396E064E678E00E94B52B83E793E083
:103C60000E944A1A87E396E06CE478E00E94B52B44
:103C700087E396E067E278E00E94B52B87E396E061
:103C80006DEF77E00E94B52B87E396E06CED77E06F
:103C90000E94B52B87E396E06FEA77E00E94B52B90
:103CA00087E396E069E877E00E94B52B87E396E02A
:103CB00065E677E00E94B52B87E396E06EE377E058
:103CC0000E94B52B87E396E00E949F2B0E94231948
:103CD0002FC087E396E061E277E028C087E396E0B3
:103CE0006CEF76E023C087E396E067EE76E01EC0D7
:103CF00087E396E068EC76E019C087E396E064E835
:103D000076E014C087E396E06FE676E00FC087E3C5
:103D100096E06AE576E00E94B52B87E396E064E1E1
:103D200076E004C087E396E06EEF75E00E94B52B65
:103D30006AE070E080E090E00E94022A04C087E31D
:103D400096E00E94AA2E87E396E00E94702E892BAF
:103D5000B1F70895A2E2B0E0E0EBFEE10C94E62FAB
:103D60008E010F5F1F4F80E1D8011D928A95E9F700
:103D700087E396E066EC71E00E942B2D0E94A81567
:103D800020E034E74BE852E32F8F38A349A35AA32E
:103D900080E09EECADEEB4E38B8F9C8FAD8FBE8F39
:103DA00024EF31E040E050E02F8B388F498F5A8F5D
:103DB00030E5C32E33ECD32EE12CF12C412C24E73B
:103DC000522E2BE8622E22E3722E8824992454016D
:103DD00033241E8A1D8A198A1A8A1B8A1C8AFFC0EC
:103DE00087E396E00E94AA2E8434B9F0853430F43B
:103DF0008332B9F18C3209F0CCC044C0833509F06C
:103E0000C8C02F8D38A149A15AA1C901DA012C01DE
:103E10003D01882499245401E2C087E396E064E4DC
:103E20000E94972B87E396E040E054E76BE872E34B
:103E30002AE030E00E94CB2C87E396E06CE20E94FF
:103E4000972B87E396E040E05EEC6DEE74E32AE0AA
:103E500030E00E94CB2C87E396E06CE20E94C92BF5
:103E6000BEC019821A821B821C821D821E821F8282
:103E7000188619861A861B861C861D861E861F8636
:103E8000188A3AC0339434E0331609F0A8C0698127
:103E90007A818B819C8128EE33E040E050E00E94E3
:103EA000772F6F8F78A389A39AA36D817E818F81ED
:103EB00098850E94772F6B8F7C8F8D8F9E8F898541
:103EC0009A85AB85BC858F8B988FA98FBA8F6D85AE
:103ED0007E858F8598890E94772F6B017C0190E207
:103EE000C9169EE4D90690E0E90690E0F90630F4A0
:103EF0008CE162E30E94BD0A332471C0A0E3CA16BC
:103F0000A5E7DA06A0E0EA06A0E0FA0618F48CE1DC
:103F100062E2F0CFB0E4CB16BCE9DB06B0E0EB0622
:103F2000B0E0FB0618F48CE166E2E4CFE0E5CE16E3
:103F3000E3ECDE06E0E0EE06E0E0FE0618F48CE1DD
:103F400062E1D8CFF0E6CF16FAEEDF06F0E0EF063A
:103F5000F0E0FF0618F48CE165E1CCCF20E7C21653
:103F600021E1D20621E0E20620E0F20618F48CE11D
:103F700061E0C0CF30EAC31636E8D30631E0E3068D
:103F800030E0F30618F48CE163E0B4CF8CE165E037
:103F9000B1CF90ED292E280E49E0421500F1032DF6
:103FA00010E0000F111F000F111F81E090E08C0F37
:103FB0009D1F080F191FD8016D917D918D919C91C6
:103FC0002AE030E040E050E00E94772F620D711D42
:103FD000811D911DF801608371838283938387E340
:103FE00096E00E94702E892B09F0FACE811491047C
:103FF000A104B10489F4C301B2010E94330B61E052
:1040000070E080E090E00E94022AFFEFFE8B1D8AA4
:10401000198A1A8A1B8A1C8A2F89388D498D5A8DD4
:1040200082169306A406B506E0F40E94DE0A2989EA
:104030003A894B895C89280F311D411D511D298BFF
:104040003A8B4B8B5C8B3D89381708F48D8B4E89EE
:10405000841708F48E8B0894811C911CA11CB11C40
:1040600056C0C301B20128EE33E040E050E00E94A8
:10407000A92F87E396E0BA01A9012AE030E00E9467
:104080005D2C87E396E06CE20E94972B87E396E035
:104090006D894AE050E00E94A52C87E396E06CE22F
:1040A0000E94972B69897A898B899C89A501940143
:1040B0000E94A92F87E396E0BA01A9012AE030E027
:1040C0000E945D2C87E396E06CE20E94972B87E3C9
:1040D00096E06E894AE050E00E94A52C87E396E0C6
:1040E0006CE20E94C92B4C0C5D1C6E1C7F1C8B8DDE
:1040F0009C8DAD8DBE8D84159505A605B70520F464
:104100004F8C58A069A07AA08824992454012F8D3F
:1041100038A149A15AA1285E33404040504009F0DF
:104120005ECFA296E2E10C940230A0E0B0E0EBE9B1
:10413000F0E20C94F12F0E94DC29611571058105D4
:104140009105C9F30E9499061092D9031092DA03DF
:104150001092DB031092DC03DD24E090D903F09091
:10416000DA030091DB031091DC03102F0F2DFE2CDE
:10417000EE240E9494062FEF30E040E050E00E94D1
:10418000CB2FE60EF71E081F191FE092D903F092FD
:10419000DA030093DB031093DC03D39444E0D416DA
:1041A000E1F6CFEDD3E000E010E040E1E42E47E29D
:1041B000F42E4EC00F5F19F40E944D084DC00E94AE
:1041C000940622E330E040E050E00E94CB2F6F5F86
:1041D000EFEDF3E090E004C08191861759F39F5F03
:1041E0009117D0F38091DE0390E08E9D90018F9D1A
:1041F000300D9E9D300D1124862F90E0AC01249F40
:10420000C001259F900D349F900D1124AA2797FD82
:10421000A095BA2F2091D5033091D6034091D703B2
:104220005091D803820F931FA41FB51F20919D03A7
:1042300030919E0340919F035091A00328173907A6
:104240004A075B0708F4B6CF69931F5F183121F066
:104250008881882309F0AECFCDB7DEB7E7E00C94B4
:104260000D3080E060E00E94FF15882331F081E08E
:1042700060E00E94FF15882341F40E9492080E948A
:104280004D080E9495200E94A5160895AAE5B0E069
:10429000ECE4F1E20C94F22F8B017A018B3009F4FB
:1042A00026C18C3040F5853009F484C0863080F416
:1042B000823009F459C0833020F4813009F050C2B3
:1042C00042C0833009F461C0843009F049C265C03E
:1042D000883009F49DC0893038F4863009F486C0EE
:1042E000873009F03DC28CC0893009F499C08A300A
:1042F00009F036C2C9C0893609F482C18A3680F411
:10430000863609F42DC1873620F4853609F028C297
:104310000EC1873609F43DC1883609F021C241C17A
:104320008C3609F4C4C18D3638F48A3609F473C169
:104330008B3609F015C2AFC18D3609F4ECC1873C4C
:1043400009F00EC200C281E069E270E00E9494119F
:1043500000ED13E0F80181918F010E947D11F3E0DF
:10436000093F1F07B9F704C282E06BE170E00E94C9
:10437000941105EB13E0F80181918F010E947D11EA
:10438000F3E0003D1F07B9F7F3C183E061E070E09F
:104390000E9494110E94FC14E9C184E061E070E085
:1043A0000E94941181E00E947D110E9476110E946A
:1043B000AA1EE0C16091210470E0660F771F85E0BE
:1043C0000E94941100E010E008C0F801EF5FFB4F7D
:1043D00080810E947D110F5F1F4F8091210490E02A
:1043E000880F991F0817190780F3C2C186E062E0A1
:1043F00070E00E94941183E793E00E948B11B8C192
:1044000087E061E070E00E94941180912204AEC1C7
:1044100088E061E070E00E94941180919B03A6C146
:1044200086E68983CE01019661E00E94DC0F0E943E
:10443000810C83E080939A0368EC70E080E090E068
:104440000E94022A80919A038430E1F48FE70E944F
:10445000930A0E94A70A8983863471F489E060E296
:1044600070E00E94941110E00E94A70A0E947D1142
:104470001F5F1032C9F77CC189E061E070E00E94E3
:104480009411C7C089E06DC18AE069E170E00E94C3
:10449000941181E080939C038091A105882351F0C1
:1044A0008091A1039091A203A091A303B091A403D2
:1044B000806809C08091A1039091A203A091A303F9
:1044C000B091A4038F778093A1039093A203A0934C
:1044D000A303B093A4030CE913E0F80181918F01C9
:1044E0000E947D11F3E0053B1F07B9F741C18BE046
:1044F00061E270E00E9494118091C0048F3F39F016
:104500008091C0048F5F8093C004815002C080916D
:10451000C0040E947D1110E0812F0E94B3110E94FF
:10452000190A0E948B111F5F1031B1F721C185E676
:1045300061E070E00E9494110932110509F015C183
:1045400020E030E0F901E053FC4FD701A20FB31F88
:104550008C9180832F5F3F4F2932310599F759C0E5
:1045600086E661E070E00E9494110B31110509F0BC
:10457000FCC020E030E0F901EB54FC4FD701A20F62
:10458000B31F8C9180832F5F3F4F2B31310599F7FB
:1045900040C087E661E070E00E9494110E94A51679
:1045A00038C088E661E070E00E94941185E78A8354
:1045B000DE011396E5EBF3E08BE101900D92815063
:1045C000E1F7CE0102966CE10E94DC0F0E94810CA3
:1045D00083E080939A0360E273E080E090E00E94C1
:1045E000022A80919A03843009F0BFC08FE70E94AD
:1045F000930A0E94A70A8A83853509F0B6C009C0CC
:1046000089E661E070E00E9494110E944D080E94CA
:10461000920881E0ABC08AE661E070E00E949411EC
:1046200089E68E8FCE014E9661E00E94DC0F0E94DB
:10463000810C83E080939A0360E273E080E090E075
:104640000E94022A80919A03843009F08EC08FE77D
:104650000E94930A0E94A70A8E8F8E01015E1F4F4F
:104660006AE3E62EF12CEC0EFD1E0E94A70AF8016B
:1046700081938F01EE15FF05C1F7A5EBB3E0FE01B5
:104680007F968BE101900D928150E1F78E8D8934F8
:1046900009F06BC0BECF8BE661E070E00E94941120
:1046A000F70180810E94C0160E943121B2CF8CE6B2
:1046B00061E070E00E9494110032110571F487E608
:1046C0008AAFDE01DB96F70180E201900D92815006
:1046D000E1F7CE01CA9661E205C087E48AAFCE0158
:1046E000CA9661E00E94DC0F0E94810C83E08093F7
:1046F0009A036CE474E080E090E00E94022A8091CA
:104700009A03843091F58FE70E94930A0E94A70ACA
:10471000873459F57ECF8DE661E070E00E949411F8
:104720000931110511F520E030E0F901E456FC4FA4
:10473000D701A20FB31F8C9180832F5F3F4F293188
:10474000310599F766CF87EC61E070E00E94941123
:1047500081E00E947D110E9476111092FF030AC031
:104760008AEC61E070E00E94941180E00E947D116B
:104770000E947611C65ADF4FE6E00C940E30A0E09E
:10478000B0E0E5ECF3E20C94EE2F84E0A82E06E016
:10479000B02E15E0C12E05E315E0B4E6DB2EA2E055
:1047A000EA2EF3E0FF2EA1C087E396E00E94AA2E36
:1047B000982F8093A00580919F05833021F184304C
:1047C00028F4813099F08230B8F409C0853009F4BA
:1047D00048C0853020F1863009F087C05FC0953B26
:1047E00009F083C081E080939F057FC0923609F075
:1047F0007AC0E0929F0579C090939E0590939D05A5
:10480000F0929F0572C090939B0510929C05809139
:104810009D05892780939D05A0929F0566C0D92F8D
:10482000C0E020919B0530919C052C2B3D2B3093B3
:104830009C0520939B0580919D05892780939D056C
:10484000C0929F052536310508F44FC08CEC61E01D
:1048500070E00E94941181E00E947D110E94761107
:1048600042C02091990530919A05F901EB5CFA4F0D
:10487000908380919D05892780939D052F5F3F4FF1
:1048800030939A052093990580919B0590919C0502
:104890002817390750F1B0929F0527C080919D05D8
:1048A000891759F46091990570919A0580919E0538
:1048B00045E355E00E9446210DC08BEC62E070E0BC
:1048C0000E94941180919E050E947D1180910004A8
:1048D0000E947D11F8018D2D11928A95E9F71092B1
:1048E0009A051092990510929F0587E396E00E9421
:1048F000702E892B09F058CFCDB7DEB7EAE00C94C3
:104900000A3081E08093FF0308C087E396E00E94AD
:10491000702E892B11F00E94BF238091FF03882302
:10492000A1F708951F93109125041F3F09F0F1C0CE
:10493000893409F467C08A3428F5883309F479C0CA
:10494000893368F4803309F486C0813308F06FC07E
:104950008B3109F44DC0813209F0D5C03DC081349E
:1049600009F49AC0823438F4893309F472C080346F
:1049700009F0C9C031C0823409F4A1C0863409F0FD
:10498000C2C052C0823609F49AC0833690F488358A
:1049900079F1893538F4823509F43FC0833509F05F
:1049A000B2C01FC08A3509F4A9C0813609F0ABC076
:1049B00073C0823791F1833730F48636A9F1893696
:1049C00009F0A1C01FC0883799F08A3709F496C052
:1049D000833709F098C005C087E396E069E471E089
:1049E00019C00E94A51687E396E063ED71E006C04A
:1049F0000E94312187E396E06DEE71E00E942B2D3D
:104A00008EEF7FC00E944D080E94920887E396E0D7
:104A10006CE072E00E942B2D76C00E94952087E307
:104A200096E065E272E0F6CF0E9443176CC08053B7
:104A300068C087E396E06CEE71E00E94B52B909120
:104A4000F803892F885F8871977E892B8093F803FC
:104A500020C089E056C087E396E069ED71E00E94CE
:104A6000B52B8091A1039091A203A091A303B091D3
:104A7000A40320E130E040E050E082279327A42700
:104A8000B5278093A1039093A203A093A303B093AF
:104A9000A4031093250437C087E396E063EC71E02C
:104AA0000E94B52B8091A1039091A203A091A30332
:104AB000B091A40320E430E040E050E012C087E36E
:104AC00096E062EB71E00E94B52B8091A10390917A
:104AD000A203A091A303B091A40320E230E040E040
:104AE00050E082279327A427B5278093A1039093B2
:104AF000A203A093A303B093A40302C00E94D31DFA
:104B00008FEF80932504809125048E3F09F4DDC04A
:104B1000D4C00E94DA16882309F4D7C080918B0490
:104B2000882321F48FEF80932504C7C086E294E0A8
:104B300060E070E040E050E00E94A2069B01AC0102
:104B400080912504992787FD9095A92FB92FFC0105
:104B50003197E930F10508F08CC0E753FF4F0C9412
:104B60001D30DA01C90181509447AB48B2438F5FD1
:104B70009945A246B24008F07CC02093D5033093FB
:104B8000D6034093D7035093D8039AC02093D903F8
:104B90003093DA034093DB035093DC0381E080938E
:104BA0008C048EC0283031054105510508F061C0E4
:104BB0002093DD0385C0DA01C9010197A109B1097C
:104BC0000A97A105B10508F054C02093DE0378C010
:104BD00086E294E06DE371E00E94BE0710E00EC033
:104BE000183130F4E12FF0E0E053FC4F87871F5F6E
:104BF00080E090E06DE371E00E94BE07009759F0FD
:104C00000E94A007009761F706C0E12FF0E0E05393
:104C1000FC4F17861F5F1831C0F352C02530310595
:104C20004105510530F52093F7034AC0DA01C90167
:104C30000197A109B1090697A105B105D0F48091AA
:104C4000F803887F822B8093F8033AC0DA01C90108
:104C50000197A109B1098050924CA140B04048F49D
:104C60002093D1033093D2034093D3035093D403C2
:104C700027C087E396E068EA71E00E942B2D13C0FD
:104C80008091D9039091DA03A091DB03B091DC030A
:104C90000196A11DB11D8093D9039093DA03A093CF
:104CA000DB03B093DC030E94D0168FEF80932504C2
:104CB00087E396E06AE00E94C92B0E94171E05C098
:104CC00080918C048823E1F2EECF1F9108958FEF3D
:104CD0008093250410928C040E94171E0CC087E359
:104CE00096E00E94702E892B31F087E396E00E94B7
:104CF000AA2E0E949224809125048E3F81F76AE0BB
:104D000070E080E090E00E94022A04C087E396E011
:104D10000E94AA2E87E396E00E94702E892BB1F79D
:104D20000895AAE2B0E0E7E9F6E20C94EB2F0E94C6
:104D3000CE297B018C0181E00E94A20B04C087E395
:104D400096E00E94AA2E87E396E00E94702E892B9F
:104D5000B1F72D98DD24D39432E6732E22E0822E13
:104D6000912C8C0E9D1E5E010894A11CB11C93E039
:104D7000C92E0E94CE2920E030E06E197F09800BF9
:104D8000910B693C71058105910510F021E030E03F
:104D90008D2D90E028233923232B99F10E94CE29D1
:104DA0007B018C012C9A80ED97E00E94E9117982B9
:104DB000D401E0EDF3E089E201900D928150E1F73A
:104DC000C5016AE20E94DC0F2C9880E090E00E940E
:104DD000E911C0929A030E94810C62E370E080E0C6
:104DE00090E00E94022A80919A03843051F4C0928C
:104DF0009A038FE70E94930A0E94A70A823409F45B
:104E0000DD248BE00E94002B892B49F5DD24D3940F
:104E100026C02D9A2C9A87E396E00E94AA2E8D3008
:104E2000910569F08E3091051CF40A97B1F407C022
:104E30008332910569F08234910579F40CC087E3DF
:104E400096E064EA71E00E94B52B0E94672605C0D7
:104E50000E94AA1E02C00E9481242D982C9887E3EC
:104E600096E00E94702E892B09F483CFD2CF8F92C7
:104E70009F92AF92BF92CF92DF92EF92FF920F93E9
:104E80001F938BE00E94002B892B09F083C068ECF4
:104E900070E080E090E00E94022A80E090E00E94B2
:104EA000E9110E94CE295B016C0140ECE42E42E145
:104EB000F42E012D112DE60EF71E081F191F06C036
:104EC0008BE00E94002B892B09F062C00E94CE2942
:104ED0006E157F058007910798F38BE00E94002BE9
:104EE000892B09F055C080ED97E00E94E9110E94DE
:104EF000CE297B018C0199249394882488E496E23E
:104F0000A0E0B0E0A80EB91ECA1EDB1E29C0AE1478
:104F1000BF04C006D10638F480ED97E00E94E91185
:104F2000882483941DC00E94CE296E197F09800BAE
:104F3000910B693C71058105910590F00E94CE2985
:104F40007B018C0180E0992009F481E0982E882370
:104F500019F480E090E002C080ED97E00E94E91132
:104F60008BE00E94002B892B91F280E090E00E9460
:104F7000E911882049F080919B038F5F83700E9424
:104F8000C0160E94312106C00E9495200E94A516DD
:104F90000E9491261F910F91FF90EF90DF90CF908C
:104FA000BF90AF909F908F90089580E06DEF77E075
:104FB00042E050E00E9409290895EF92FF920F937A
:104FC0001F9380E00E9419080E94D4118DE061E0D7
:104FD0000E94612A8CE061E00E94612A8BE060E01F
:104FE0000E94612A83E060E00E94612A83E061E020
:104FF0000E94CD2A8EE061E00E94612A8EE060E08E
:105000000E94CD2A0E94D41487E396E040E052EC3F
:1050100061E070E00E94E92D0E94B3160E943121E8
:105020000E94770D8FEF8093C0040E94D52778945B
:105030000E94CE297B018C018091C0048F3F09F032
:10504000DEC00E94CE296E197F09800B910B605D36
:1050500077408040904008F0D2C0EECF87E396E0E2
:105060000E94AA2E87E396E00E94702E892BB1F74A
:1050700087E396E062E472E00E94282D83E793E0E4
:105080000E944A1A87E396E069E572E00E94282DA3
:1050900087E396E062E070E04AE050E00E94142D61
:1050A00062E370E080E090E00E94022A87E396E0ED
:1050B0000E94702E04970CF187E396E00E94AA2EBE
:1050C00082349105D1F487E396E00E94AA2E8E34B3
:1050D000910599F487E396E00E94AA2E8434910505
:1050E00061F487E396E00E94AA2E819731F480E074
:1050F00090E00E94E9110E9491264091D1035091C5
:10510000D2036091D3037091D403DB01CA010197EC
:10511000A109B1090497A105B10568F44093C10440
:10512000433029F040E052EC61E070E004C040EA16
:1051300056E861E070E087E396E00E94E92D0E9466
:1051400037272D9880E090E00E94E9110E94770DAA
:105150001092A5048091A10383FF11C08091E50303
:10516000882351F08091EC03882331F08091F30380
:10517000882311F087E001C085E08093A50480E0DA
:105180000E94A20B8091A4040E94C80A0E94810C74
:105190001092290510922A0510922B0510E015C0D7
:1051A00062E370E080E090E00E94022A80ED97E0E8
:1051B0000E94E91162E370E080E090E00E94022A20
:1051C00080E090E00E94E9111F5F80919B038117AE
:1051D00038F78091F80390E084FF09C020E08871DF
:1051E0009070489709F421E0822F0E94DD148FE02F
:1051F0000E9419081F910F91FF90EF90089580ED84
:1052000097E00E94E9118BE061E00E94CD2A2D9A7F
:1052100029CF823000F5E82FF0E0EE0FFF1FEE55AA
:10522000FA4F71836083882319F08130A1F408C09C
:10523000809169008C7F842B80936900E89A08959F
:1052400080916900440F551F440F551F837F842BA5
:1052500080936900E99A08951F920F920FB60F92FA
:1052600011242F933F934F935F936F937F938F936B
:105270009F93AF93BF93EF93FF938091A20590917B
:10528000A305892B29F0E091A205F091A3050995CA
:10529000FF91EF91BF91AF919F918F917F916F910E
:1052A0005F914F913F912F910F900FBE0F901F90E4
:1052B00018951F920F920FB60F9211242F933F93C0
:1052C0004F935F936F937F938F939F93AF93BF930E
:1052D000EF93FF938091A4059091A505892B29F068
:1052E000E091A405F091A5050995FF91EF91BF917B
:1052F000AF919F918F917F916F915F914F913F916E
:105300002F910F900FBE0F901F9018951F920F9224
:105310000FB60F9211242F933F938F939F93AF93C8
:10532000BF938091AA059091AB05A091AC05B09177
:10533000AD053091AE050196A11DB11D232F2D5F46
:105340002D3720F02D570196A11DB11D2093AE05DC
:105350008093AA059093AB05A093AC05B093AD05DF
:105360008091A6059091A705A091A805B091A905E7
:105370000196A11DB11D8093A6059093A705A0934A
:10538000A805B093A905BF91AF919F918F913F91CF
:105390002F910F900FBE0F901F9018958FB7F89414
:1053A0002091AA053091AB054091AC055091AD0517
:1053B0008FBFB901CA0108959FB7F8942091A6053F
:1053C0003091A7054091A8055091A90586B5A89BE5
:1053D00006C08F3F21F02F5F3F4F4F4F5F4F9FBF62
:1053E000542F432F322F2227280F311D411D511DCD
:1053F00082E0220F331F441F551F8A95D1F7B90150
:10540000CA010895EF92FF920F931F93CF93DF93FA
:105410007B018C010E94DC29EB010EC00E94DC297B
:105420006C1B7D0B685E7340C8F30894E108F108BB
:1054300001091109C851DC4FE114F10401051105FE
:1054400069F7CDB7DEB7E6E00C940E30789484B5FA
:10545000826084BD84B5816084BD85B5826085BD70
:1054600085B5816085BDEEE6F0E080818160808356
:10547000E1E8F0E010828081826080838081816039
:105480008083E0E8F0E0808181608083E1EBF0E000
:10549000808184608083E0EBF0E0808181608083A4
:1054A000EAE7F0E08081846080838081826080838D
:1054B0008081816080838081806880831092C100B8
:1054C0000895CF93DF93482F50E0CA018D5F934F2B
:1054D000FC0134914151544FFA018491882369F1C0
:1054E00090E0880F991FFC01EF52F44FA591B49101
:1054F000FC01E552F44FC591D491662351F42FB7C6
:10550000F8948C91932F909589238C93888189238B
:105510000BC0623061F42FB7F8948C91932F909563
:1055200089238C938881832B88832FBF06C09FB7E4
:10553000F8948C91832B8C939FBFDF91CF9108952A
:10554000833071F0843028F48130A1F0823021F56D
:1055500014C08630B1F08730D1F08430E9F404C053
:10556000809180008F7703C0809180008F7D809331
:105570008000089584B58F7702C084B58F7D84BD87
:1055800008958091B0008F778093B0000895809146
:10559000B0008F7D8093B0000895FF920F931F930A
:1055A000F62E482F50E0CA01895E934FFC012491EA
:1055B000CA018D5F934FFC0114914151544FFA0180
:1055C00004910023C9F0222319F0822F0E94A02AFF
:1055D000E02FF0E0EE0FFF1FE552F44FA591B491DC
:1055E0009FB7F894FF2021F48C911095812302C07D
:1055F0008C91812B8C939FBF1F910F91FF900895E9
:105600000F931F93482F50E0CA01895E934FFC010E
:105610002491CA018D5F934FFC0104914151544F75
:10562000FA011491112319F420E030E015C022236F
:1056300019F0822F0E94A02A812F90E0880F991FD5
:105640008B51944FFC01A591B4918C9120E030E0F6
:10565000802311F021E030E0C9011F910F910895DE
:10566000982F8E3008F09E50977080914803829555
:10567000880F880F807C892B80937C0080917A0032
:10568000806480937A0080917A0086FDFCCF20911F
:10569000780040917900942F80E030E0282B392B5E
:1056A000C9010895A0E0B0E0E8E5FBE20C94F02F1A
:1056B0007C016B018A01C0E0D0E00FC0D6016D9182
:1056C0006D01D701ED91FC910190F081E02DC701B2
:1056D0000995C80FD91F015010400115110571F728
:1056E000CE01CDB7DEB7E8E00C940C30EF92FF921C
:1056F0000F931F93CF93DF937C018B01C0E0D0E029
:10570000F8010F5F1F4F6491662359F0D701ED91A7
:10571000FC910190F081E02DC7010995C80FD91FB8
:10572000EFCFCE01CDB7DEB7E6E00C940E30DC0152
:10573000ED91FC910190F081E02D09950895EF9293
:10574000FF920F931F938C016DE00E94972B7C01B9
:10575000C8016AE00E94972B9C012E0D3F1DC901D4
:105760001F910F91FF90EF900895EF92FF920F938A
:105770001F937C010E94762B8C01C7010E949F2BF6
:105780009C01200F311FC9011F910F91FF90EF90D5
:105790000895EF92FF920F931F937C010E94972B25
:1057A0008C01C7010E949F2B9C01200F311FC90152
:1057B0001F910F91FF90EF900895CF93DF93EC012D
:1057C0006115710519F420E030E00FC0DB010D9088
:1057D0000020E9F71197A61BB70BE881F981028039
:1057E000F381E02DAD0109959C01C901DF91CF91B5
:1057F00008954F925F927F928F929F92AF92BF9245
:10580000CF92DF92EF92FF920F931F93DF93CF938C
:10581000CDB7DEB7A1970FB6F894DEBF0FBECDBFF0
:105820002C01742ECB01223008F42AE019A231E2B7
:10583000C32ED12CCC0EDD1E822E9924AA24BB248B
:10584000672D752FA50194010E94A92F79018A0166
:10585000C801B701A50194010E94772F472D461B6F
:105860000894C108D1084A3010F4405D01C0495C79
:10587000F6014083E114F1040105110521F07E2CAD
:105880005F2DC801DDCFC201B6010E94DD2BA196BC
:105890000FB6F894DEBF0FBECDBFCF91DF911F9141
:1058A0000F91FF90EF90DF90CF90BF90AF909F90BF
:1058B0008F907F905F904F900895DC012115310506
:1058C00041F4ED91FC910190F081E02D642F099558
:1058D00008950E94F92B0895EF92FF920F931F9362
:1058E0007C010E945D2C8C01C7010E949F2B9C01B2
:1058F000200F311FC9011F910F91FF90EF90089564
:10590000EF92FF920F931F939A017B0100E010E04A
:10591000B801A7010E945D2C1F910F91FF90EF909D
:105920000895EF92FF920F931F937C010E94802CA9
:105930008C01C7010E949F2B9C01200F311FC901C0
:105940001F910F91FF90EF900895EF92FF920F93A8
:105950001F939A01E62EFF2400E010E0B801A70192
:105960000E945D2C1F910F91FF90EF900895EF9290
:10597000FF920F931F937C010E94A52C8C01C701FD
:105980000E949F2B9C01200F311FC9011F910F9175
:10599000FF90EF900895A0E0B0E0E1EDFCE20C9400
:1059A000F02FEC016A017B012115310541F4E881FA
:1059B000F9810190F081E02D642F09951BC02A30F8
:1059C0003105B1F477FF13C06DE20E94972B8C0173
:1059D00044275527BA014C195D096E097F09CE018C
:1059E0002AE00E94F92B9C01200F311F04C02AE0FD
:1059F0000E94F92B9C01C901CDB7DEB7E8E00C94F9
:105A00000C30EF92FF920F931F937B019A010027B6
:105A1000F7FC0095102FB801A7010E94CB2C1F9115
:105A20000F91FF90EF900895EF92FF920F931F93C5
:105A30007C010E94012D8C01C7010E949F2B9C01BB
:105A4000200F311FC9011F910F91FF90EF90089512
:105A50000E94DD2B0895EF92FF920F931F937C011C
:105A60000E94282D8C01C7010E949F2B9C01200FB2
:105A7000311FC9011F910F91FF90EF900895089574
:105A80001F920F920FB60F9211242F933F934F93B3
:105A90008F939F93EF93FF938091C00082FD1DC071
:105AA0004091C6002091EF053091F0052F5F3F4FE8
:105AB0002F7330708091F1059091F2052817390706
:105AC00071F0E091EF05F091F005E155FA4F408358
:105AD0003093F0052093EF0502C08091C600FF913E
:105AE000EF919F918F914F913F912F910F900FBE0A
:105AF0000F901F9018951F920F920FB60F921124BE
:105B00002F933F938F939F93EF93FF9320913306AF
:105B10003091340680913506909136062817390762
:105B200031F48091C1008F7D8093C10014C0E09159
:105B30003506F0913606ED50FA4F208180913506FA
:105B40009091360601968F739070909336068093ED
:105B500035062093C600FF91EF919F918F913F9161
:105B60002F910F900FBE0F901F901895A0E0B0E0FE
:105B7000ECEBFDE20C94EC2FFC011382128288EE18
:105B800093E0A0E0B0E084839583A683B7838BE89D
:105B900093E0918380837587648757874687318B2D
:105BA000208B138B028BF58AE48AD78AC68AB18E42
:105BB000A08E938E828E8F85848F8889858F898928
:105BC000868F8A89878F8B8980A32096ECE00C943E
:105BD0000830AF92BF92DF92EF92FF920F931F9324
:105BE000CF93DF93EC017A018B01DD24403081EE0D
:105BF000580780E0680780E0780711F0DD24D3942F
:105C000091E0A92EB12CEC89FD89DD2069F0C50158
:105C100008A002C0880F991F0A94E2F7808360E011
:105C200079E08DE390E005C0108260E874E88EE1D1
:105C300090E0A80197010E94A92F215030404040D8
:105C40005040569547953795279580E12030380785
:105C500020F0DD2011F0DD24D6CFE889F9893083EA
:105C6000EA89FB89208319A2EE89FF89408121E01E
:105C700030E0C9010C8C02C0880F991F0A94E2F72A
:105C8000482B4083EE89FF894081C9010D8C02C0F9
:105C9000880F991F0A94E2F7482B4083EE89FF8909
:105CA0004081C9010E8C02C0880F991F0A94E2F747
:105CB000482B4083EE89FF8980810F8C02C0220F20
:105CC000331F0A94E2F7209528232083DF91CF9198
:105CD0001F910F91FF90EF90DF90BF90AF900895CC
:105CE000DC011C96ED91FC911D97E05CFF4F21912A
:105CF000319180819181281B390B2F733070C9013C
:105D0000089587E396E00E94702E892B11F00E947F
:105D10003F2D0895DC011C96ED91FC911D97E05CF0
:105D2000FF4F20813181E054F040DF01AE5BBF4F77
:105D30008D919C9111972817390719F42FEF3FEF98
:105D400007C08D919C91E80FF91F8081282F30E0CA
:105D5000C9010895DC011C96ED91FC911D97E05C52
:105D6000FF4F20813181E054F040DF01AE5BBF4F37
:105D70008D919C9111972817390719F42FEF3FEF58
:105D800010C08D919C911197E80FF91F20818D9182
:105D90009C91119701968F73907011969C938E939E
:105DA00030E0C9010895DC0191968C919197882388
:105DB00039F05496ED91FC915597808186FFF9CF8B
:105DC00091961C920895CF93DF93EC01EE85FF85A9
:105DD000E05CFF4F20813181E054F0402F5F3F4F66
:105DE0002F733070DF01AE5BBF4F8D919C91119787
:105DF00028173907D1F3E05CFF4F80819181E0548F
:105E0000F040E80FF91F6083EE85FF85E05CFF4FEF
:105E100031832083EE89FF89208181E090E00F8C1F
:105E200002C0880F991F0A94E2F7282B208381E093
:105E300089A3EC89FD8980818064808381E090E082
:105E4000DF91CF9108958F929F92AF92BF92CF92A0
:105E5000DF92EF92FF920F931F9300D000D00F922A
:105E6000EDB7FEB7319684E0ADB7BEB711968C930F
:105E700083E0818387E0828385E0838381E084837C
:105E800087E396E06FEA75E043EF55E025EC30E0FC
:105E900004EC10E0B0ECEB2EF12CA1ECCA2ED12CCE
:105EA000F2ECAF2EB12CE6EC8E2E912C0E94B62D8A
:105EB0000F900F900F900F900F901F910F91FF90E8
:105EC000EF90DF90CF90BF90AF909F908F9008950C
:105ED000CF93DF930E94262A0E94DD27C1E8DEE2ED
:105EE0000E94F3112097E1F30E94812EF9CF629F67
:105EF000D001739FF001829FE00DF11D649FE00DC2
:105F0000F11D929FF00D839FF00D749FF00D659F22
:105F1000F00D9927729FB00DE11DF91F639FB00D21
:105F2000E11DF91FBD01CF011124089597FB092E32
:105F300007260AD077FD04D086D006D000201AF4B8
:105F4000709561957F4F0895F6F7909581959F4FD5
:105F50000895A1E21A2EAA1BBB1BFD010DC0AA1FAA
:105F6000BB1FEE1FFF1FA217B307E407F50720F0C2
:105F7000A21BB30BE40BF50B661F771F881F991F3D
:105F80001A9469F760957095809590959B01AC0186
:105F9000BD01CF01089597FB092E05260ED057FDB0
:105FA00004D0D7DF0AD0001C38F4509540953095C6
:105FB00021953F4F4F4F5F4F0895F6F7909580958D
:105FC000709561957F4F8F4F9F4F08952F923F920D
:105FD0004F925F926F927F928F929F92AF92BF92F9
:105FE000CF92DF92EF92FF920F931F93CF93DF93A5
:105FF000CDB7DEB7CA1BDB0B0FB6F894DEBF0FBE02
:10600000CDBF09942A88398848885F846E847D844E
:106010008C849B84AA84B984C884DF80EE80FD8050
:106020000C811B81AA81B981CE0FD11D0FB6F894C6
:10603000DEBF0FBECDBFED010895EE0FFF1F05902F
:10604000F491E02D0994AA1BBB1B51E107C0AA1FC4
:10605000BB1FA617B70710F0A61BB70B881F991F09
:106060005A95A9F780959095BC01CD01089591119D
:1060700006C0803219F089508550D0F708959927CD
:0860800088270895F894FFCF72
:106088004E6F005965730054582074696D656F75BB
:106098007421006D6F64756C65206C6F636B65644B
:1060A8003F00486F70206368616E6E656C20002049
:1060B80040200053004E2F4100386368002C002C0C
:1060C800205B005D20280029004E4F5420454E419A
:1060D800424C45440053656E64696E67207365746D
:1060E80074696E677320746F2052580A0052657382
:1060F800657474696E672073657474696E6773205C
:106108006F6E2052580A0041626F72746564206590
:10611800646974730A00696E76616C6964207365DA
:106128006C656374696F6E000D0A496E76616C69FF
:106138006420696E707574202D20646973636172C0
:106148006465642107007363616E6E6572206D6F0C
:1061580064650053657474696E677320736176654E
:106168006420746F20454550524F4D0A00526576A1
:1061780065727465642073657474696E67732066EC
:10618800726F6D20454550524F4D0A004C6F616447
:10619800656420666163746F7279206465666175F1
:1061A8006C74730A004B657920616E6420636861C2
:1061B8006E6E656C732072616E646F6D697A65646A
:1061C8000A004F70656E4C52536E67205458207306
:1061D80074617274696E672000206F6E20485720C2
:1061E8000050504D0052535349005344410053430B
:1061F8004C00525844005458440041494E004C4207
:106208004545500053504B54524D0053425553008E
:1062180053554D44004C4C494E440000342B340037
:106228003800382B340031320031322B340031360B
:106238000001000000C01200001A400AA1204EA56B
:10624800001B1E27522C23308025000005400AA180
:10625800204EA50020244EA52C2330004B0000061C
:10626800400AD0009D49007B289D492C233000E13D
:10627800000005400A4501D7DC03B81E0EBF002305
:106288002E48E801008A400A6001555502AD1E20DB
:10629800000023C88025000005400AA1204EA50063
:1062A80020244EA52C233000020002000200020028
:1062B80002000200020002000200020002000200C6
:1062C80002000200020002FF01610265026A026E1A
:1062D80002720276027A027E0284028B0290029592
:1062E800029B029B029B029B0235019C02A002A218
:1062F80002A602A902AE02350100070B0C10111507
:1063080000160A1322312900000000E32E522B70D8
:086318002EAA2E8A2ED32E00BE
:107E00000F92CDB7DEB7112484B714BE81FFF1D035
:107E100082E08093C00088E18093C10086E0809377
:107E2000C20080E18093C4008EE0CDD088249924E4
:107E3000CC24C394F5E0DF2EE1E1EE2E73E0F72EC3
:107E4000B6D0082F813479F4B2D08983C2D0898129
:107E5000823811F481E005C0813811F485E001C059
:107E600083E09ED09AC0823411F484E103C085344B
:107E700019F485E0B6D091C0853561F498D0082F0B
:107E800010E095D090E0982E8824802A912A880CC2
:107E9000991C82C0863521F484E0A3D080E0E1CF34
:107EA000843609F04CC083D082D0A82E80D0B82E62
:107EB00000E011E07CD0F80181938F01AE16D1F77C
:107EC00088D0FB2DF53489F4E0E0F1E00BC0F9999E
:107ED000FECF92BC81BC0894811C911C819180BD15
:107EE000FA9AF99AEA1598F358C08B2D863409F05E
:107EF00054C0F401F7BEE89507B600FCFDCFF401CD
:107F0000A0E0B1E02C9130E011968C91119790E0B7
:107F1000982F8827822B932B12960C01C7BEE895C9
:107F20001124329681E0A038B80761F7F401D7BE7A
:107F3000E89507B600FCFDCFE7BEE8952EC0843774
:107F4000F1F435D034D0182F32D0B82E42D0FB2DDA
:107F5000F63421F4F40105914F010CC0FB2DF534EA
:107F600049F4F999FECF92BC81BC0894811C911C04
:107F7000F89A00B5802F14D0115049F70EC08537FC
:107F800039F427D08EE10CD085E90AD08FE069CF93
:107F9000813511F488E017D01CD080E101D050CF9A
:107FA0009091C00095FFFCCF8093C600089580910A
:107FB000C00087FFFCCF8091C00084FD01C0A89560
:107FC0008091C6000895E0E6F0E098E19083808318
:107FD0000895EDDF803219F088E0F5DFFFCF84E10E
:107FE000DFCF1F93182FE3DF1150E9F7F2DF1F9166
:0E7FF0000895282E80E0E7DFEE27FF27099492
:027FFE0001057B
:0400000300007E007B
:00000001FF
